:0800000083011F308A00042F68
:103E0800203084004E300F2783010A168A15332F7D
:103E180004068001840A0406031D0C2F0034831253
:103E28000313CB000C1E162F4B08990008003030E6
:103E380083120313CB001230CC007A30CD00CD08AA
:103E480003192F2F6400CC080319CD03CC038C1E53
:103E5800232F1A080800CB0B1F2F003008008316E9
:103E68000313860164004030990024309800903094
:103E78008312980086011B27E33A03194C2F093A4D
:103E880003194A2F073A0319EA2FF72FEB30E82FC7
:103E98001B27A700A6011B27A6041B27A0001B277A
:103EA800A200A301A101200823020318692F2308F7
:103EB800283E840083131B2780002308283E8400A3
:103EC80083130008A107A30A572F21082206031904
:103ED8006F2FE830E82FE7301327A301CB2F2030CE
:103EE80027020318E12F831603178C177E2F8316DA
:103EF80003178C13831203132308283E84008313AB
:103F0800000803178E000E080313C900230A283E71
:103F180084008313000803178C000C080313C800DF
:103F2800260803178D0000300313270204300319F5
:103F380026020318A12F1F30A22F270803178F006E
:103F480003130D12831603170C1555308D00AA3074
:103F58008D008C1400000000831203132708213AF7
:103F6800031DB92F0D1EB62F0D12831603170C1142
:103F78000C140000000083120E0803134906031DE9
:103F8800CB2F03170C08031348060319E12F200849
:103F980023020318E72F2708213A03197B2F1F3024
:103FA80027020430031926022030031C742F27022D
:103FB8000030031926020318732F0230A307A60A3C
:103FC8000319A70ACB2FE43013273F2FE430132718
:103FD8001830CA00FA30A4000000A40BF02FCA035E
:103FE800CA08031DEE2F0230831698008312980129
:063FF8000A168A15002FD5
:02400E00723FFF
:00000001FF
